:1000000083177D3084007E300A128A110D200A1277
:100010008A1183010A128A11152864008001840A5A
:1000200004060319003404060E2803108316031374
:100030000030031801308500803087000310003045
:1000400003180130880003108312031300300318D3
:10005000013088000F3085000A128A11F5230A1238
:100060008A110030831203179F000030A000382847
:10007000FA300A128A1116240A128A1183120317FF
:1000800001309F070318A00A0030A0072008803A1B
:10009000D10080305102031D4F2802301F02031C83
:1000A0005228532838280D300A128A1104240A12C3
:1000B0008A110A300A128A1104240A128A11EC30B9
:1000C00083120317D4000630D5000A128A11302497
:1000D0000A128A1183120313071087100711871160
:1000E0000030831203179D0000309E007D10003009
:1000F0009300003094000F309700003098001930C2
:10010000B9000A30D1005108BA001230D1005108AC
:10011000BB001730D1005108BC000E30D10051088F
:10012000BD001530D1005108BE002430D100510867
:10013000BF001630D1005108C0001C30D10051085A
:10014000C1001030D1005108C2002430D100510844
:10015000C3000A30D1005108C4001B30D10051083F
:10016000C5001730D1005108C6000E30D10051082B
:10017000C700140813040319BE28BF2846290030FD
:100180009F000030A00026291F08213E831784000D
:1001900030300002031CCD28CE28DC281F08213E69
:1001A00084003A3000020318D628D728DC283030E3
:1001B0009B0000309C0015291F08213E840041301F
:1001C0000002031CE428E528F3281F08213E8400D0
:1001D0005B3000020318ED28EE28F32837309B002F
:1001E00000309C0015291F08213E84006130000268
:1001F000031CFB28FC280A291F08213E84007B30B1
:1002000000020318042905290A2957309B000030F1
:100210009C0015292430D1001F08213E840051087C
:10022000800000309B0000309C001F08213E8400AD
:100230001B080002D1001F08393E840051088000CD
:1002400001309F070318A00A0030A0071D08013ED7
:10025000D1001E080318013E003ED2002008803A5B
:10026000D3005208803A5302031D382951081F0257
:10027000031C3B293C29C4281E08980198071D0827
:100280009701970700309300003094001808D701B9
:10029000D7071708D601D6071430D4000030D50090
:1002A0000A128A117E240A128A1183120317550832
:1002B0009A019A075408990199071A08803AD100BF
:1002C00080305102031D6629023019020318692982
:1002D0006A297B291808803AD10080305102031D19
:1002E00073290C3017020318762977297B290230ED
:1002F000990000309A001A08803AD10080305102EB
:10030000031D8429013019020318872988298C29A3
:100310000130990000309A0000309F000030A000AA
:10032000E42A00309B0000309C00D02A0030950069
:1003300000309600BC2A0530E4000030E5001608C5
:10034000E301E3071508E201E2070A128A115424C7
:100350000A128A118312031762081F02D40063086D
:10036000031C630A2002D5001508393E8317840058
:1003700000080A128A11F2240A128A118312031346
:100380008C1EC329C429B42A0A128A11F5270A121D
:100390008A11831203179000A92A0D300A128A11BC
:1003A00004240A128A110A300A128A1104240A1239
:1003B0008A11831203171E08803AD100803051023F
:1003C000031DE42901301D02031CE729E8291E2A28
:1003D0002E30D4000730D5000A128A1130240A12B8
:1003E0008A110030831203179100003092000A2A0C
:1003F0001108213E8317840000080A128A11042480
:100400000A128A1183120317013091070318920A06
:10041000003092071208803AD1001E08803A51023B
:10042000031D142A1D081102031C172A182AF82973
:100430007D1001309300003094002E2AC530D40086
:100440000630D5000A128A1130240A128A117D1052
:10045000003083120317930000309400B42A100870
:100460000A128A1104240A128A1183120317FF3018
:100470009D0703189E0AFF309E079E1F402A412AAF
:10048000452A00309D0000309E00B42A7D140030C3
:100490009D0000309E000D300A128A1104240A12B9
:1004A0008A110A300A128A1104240A128A1144306D
:1004B00083120317D4000730D5000A128A113024A2
:1004C0000A128A11B42A7D1C662A672AA82A1830C3
:1004D0001D061E04031D6D2A6E2A922A0D300A1273
:1004E0008A1104240A128A110A300A128A11042479
:1004F0000A128A110F3083120317D4000730D50077
:100500000A128A1130240A128A110D300A128A1135
:1005100004240A128A110A300A128A1104240A12C7
:100520008A11A82A10080A128A1104240A128A11B0
:10053000831203171008D1001D08213E8317840081
:100540005108800001309D0703189E0A00309E0765
:10055000B42A1008083A03192F2A053A0319CD299D
:10056000F33A0319462A632A8312031701309507C9
:100570000318960A003096071608803AD10018082A
:10058000803A5102031DC62A17081502031CC92A06
:10059000CA2A9B2901309B0703189C0A00309C073C
:1005A0001C08803AD1001A08803A5102031DDA2A49
:1005B00019081B02031CDD2ADE2A962901309F0739
:1005C0000318A00A0030A0070530E4000030E50061
:1005D0001808E301E3071708E201E2070A128A118B
:1005E00054240A128A118312031762083C3ED10078
:1005F00063080318013E003ED2002008803AD30071
:100600005208803A5302031D072B51081F02031C96
:0E0610000A2B0B2B9129B9280A128A110028F7
:1007EA00193083160313990024309800903083122D
:1007FA00031398008316031307138717080083123D
:10080A000317DA00092C092C831203130C1E0E2C71
:10081A000F2C082C831203175A088312031399000A
:10082A000800D4000430D5005330D6001D2C1D2CEE
:10083A000130D602031D222C232C1C2C0130D50298
:10084A00031D282C292C192C0130D402031D2E2C0F
:10085A002F2C172C08005630D7003A2C56080A12AB
:10086A008A1104240A128A113A2C83120317550892
:10087A00D9005408D8000130D4070318D50A5808FB
:10088A00840059080A128A1100260A128A11D6000F
:10089A00D608031D512C522C332C532C080000303F
:1008AA00E6000030E700621C5B2C5C2C622C6408BA
:1008BA00E6070318E70A6508E70701300310E40DA5
:1008CA00E50DFF3E031D632C01300310E30CE20C1F
:1008DA00FF3E031D6A2C63086204031D752C762CE7
:1008EA00582C6708E301E3076608E201E2077D2C5A
:1008FA0008000310003003180130D900D71F862CD6
:10090A00872C8F2CD609D709D60A0319D70AD901F9
:10091A000314D90DD51F922C932C9C2CD409D509DC
:10092A00D40A0319D50A0130DC005C08D906003064
:10093A00DA000030DB00570856040319A52CA62C50
:10094A00E12CD8010314D80DB52C01300310D60DB3
:10095A00D70DFF3E031DAB2C0130DC005C08D80725
:10096A00D71FB82CB92CAA2C01300310DA0DDB0DD5
:10097A00FF3E031DBA2C57085502031DC62C560804
:10098A005402031CC92CCA2CD42C5608D40257086A
:10099A00031CD503D5020130DA040030DB04013030
:1009AA000310D70CD60CFF3E031DD52C0130D802FC
:1009BA00031DE02CE12CB92CD908031DE52CEA2CE7
:1009CA00DA09DB09DA0A0319DB0A5B08D501D5075C
:1009DA005A08D401D407F12C0800D6000030D900F7
:1009EA000030DA000030D7000030D8000030DB00D9
:1009FA000030DC00002D0530E4000030E500560828
:100A0A00DE00DF015E08E2005F08E3000A128A11D5
:100A1A0054240A128A11831203175B086207E00042
:100A2A005C0803185C0A6307E1000C306007840065
:100A3A0006300318073061070A128A1100260A12C3
:100A4A008A11831203138800831203175908540268
:100A5A00D7005A08031C5A0A5502D8005808E3015D
:100A6A00E3075708E201E2070A128A116A250A1205
:100A7A008A11093083120317DD00442D442D0130F9
:100A8A00DD02031D492D4A2D432D0F308312031316
:100A9A008500831203170130D9070318DA0A0030D8
:100AAA00DA070130DB070318DC0A0030DC075C08D0
:100ABA00803ADE0080305E02031D652D05305B0240
:100ACA00031C682D692D002D08006308803AE70091
:100ADA0080306702031D732D103062020318762DD1
:100AEA00772D7E2D0E30E5000030E6006208E40026
:100AFA00ED2D6308803AE70080306702031D872DD9
:100B0A0010306202031C8A2D8B2DA02D6308803AB7
:100B1A00E70080306702031D942D2030620203181B
:100B2A00972D982DA02D0D30E5000030E6006208C3
:100B3A00F03EE400ED2D6308803AE700803067025A
:100B4A00031DA92D20306202031CAC2DAD2DC22D30
:100B5A006308803AE70080306702031DB62D303003
:100B6A0062020318B92DBA2DC22D0B30E5000030F0
:100B7A00E6006208E03EE400ED2D6308803AE700F3
:100B8A0080306702031DCB2D30306202031CCE2D4C
:100B9A00CF2DE42D6308803AE70080306702031DF9
:100BAA00D82D3C3062020318DB2DDC2DE42D0730F2
:100BBA00E5000030E6006208D03EE400ED2D0F307B
:100BCA00E5000030E6000310003003180130E400AD
:100BDA006408E700E8016708E9006808EA000A1201
:100BEA008A1158270A128A11831203176508831279
:100BFA00031385000800FE00FE1F082E83137E18CB
:100C0A008317000808008A000408820000343E3472
:100C1A005134493445343E340434023401347F3487
:100C2A00003472344934493449344634223449341C
:100C3A004934493436340C340A34093409347F349B
:100C4A004F3449344934493431343E3449344934CF
:100C5A0049343234413421341134093407343634B6
:100C6A0049344934493436340634093409340934A8
:100C7A007E347C341234113412347C347F34493457
:100C8A004934493436343E344134413441342234CF
:100C9A007F344134413441343E347F344934493419
:100CAA00493441347F3409340934093401343E3437
:100CBA004134493449343A347F34083408340834E6
:100CCA007F34413441347F344134413471344134C6
:100CDA007F34013401347F340834143422344134EB
:100CEA007F3440344034403440347F340234043456
:100CFA0002347F347F340234043408347F343E347F
:100D0A004134413441343E347F340934093409349E
:100D1A0006343E344134513461343E347F3409342C
:100D2A00193429344634263449344934493432345E
:100D3A00013401347F34013401343F3440344034C7
:100D4A0040343F341F342034403420341F347F343D
:100D5A002034103420347F34633414340834143487
:100D6A00633441342234143408340734613451343E
:100D7A0049344534433400340034003400340034F8
:100D8A004D3465346E3473346134673465346D348C
:100D9A002034763461347A3469346134213421342C
:100DAA00213420344D3461346E34743465346E34F5
:100DBA0064346F3420346134203461346E347434D2
:100DCA006934673461342134213421340034503495
:100DDA00613469346E3465346C3420346434653477
:100DEA0020346D3465346E34733461346734653459
:100DFA006E34733420342D343E3420346F347034DE
:100E0A006534723461346E3464346F34213421347D
:100E1A0021340034423475346634663465347234AD
:100E2A00203463346834653469346F3421342134AE
:100E3A00213420345434653463346C3465342034BA
:100E4A0045344E3454344534523421342134213417
:100E5A0000344D3465346E34733461346734653428
:100E6A006D342034723465346334653462346934E1
:100E7A006434613420342D343E34203400340A344E
:100E8A0045346E3476346934653420346134203420
:100E9A006D3465346E3473346134673465346D345B
:100EAA002D343E34003483120313071087100711C0
:100EBA008711BA2F8312031307108710071187119E
:100ECA00F42F831203130714F42F831203138714C6
:100EDA00F42F8312031307148714F42F83120313B6
:100EEA000715F42F8312031307140715F42F83121F
:100EFA00031387140715F42F831203130714871497
:100F0A000715F42F831203138715F42F8312031383
:100F1A0007148715F42F8312031387148715F42FE8
:100F2A0083120313071487148715F42F83120313EC
:100F3A0007158715F42F831203130714071587154E
:100F4A00F42F83120313871407158715F42F8312BE
:100F5A0003130714871407158715F42F8312031335
:100F6A000710871007118711F42F83120317EF2F29
:100F7A006908003A03195F2F013A0319662F033AE9
:100F8A0003196A2F013A03196E2F073A0319732FAF
:100F9A00013A0319772F033A03197C2F013A0319EF
:100FAA00812F0F3A0319872F013A03198B2F033A1E
:100FBA000319902F013A0319952F073A03199B2F0A
:100FCA00013A0319A02F033A0319A62F013A03196C
:100FDA00AC2FB32F6A08003A0319BD2FB32F0800AC
:100FEA00F72FF72F8C1EFA2FFB2FF62F1A08FD2F3B
:020FFA000800ED
:00000001FF
